:020000040800F2
:10500000501A0020D550000871820008817A0008EB
:105010000000000000000000000000000000000090
:10502000000000000000000000000000B98F000830
:10503000000000000000000095880008CD900008E6
:10504000E7500008E7500008E7500008E750000864
:10505000E7500008295B0008E7500008E750000807
:1050600000000000E7500008515A0008E75000080F
:10507000E7500008ED7E000800000000E75000083F
:1050800000000000E75000080000000000000000E1
:10509000E750000800000000E7500008E750000853
:1050A000E7500008E7500008E75000085D98000846
:1050B000E7500008E7500008000000000000000072
:1050C0000348854600F060FC0048004771A60008D0
:1050D000501A00200448804704480047FEE7FEE7D6
:1050E000FEE7FEE7FEE7FEE769910008C150000811
:1050F00030B50B46014600202022012409E00D4670
:10510000D5409D4205D31D469540491B25469540F7
:1051100040191546521E002DF1DC30BDF0B51FB40C
:105120000646002082B005464024019100901BE015
:10513000019922460F46304600F04EFB049A059B2B
:10514000801A994110D310461946224600F034FBCC
:10515000361A8F410197224601200021009F00F05E
:105160002BFB38184D4100902046641E0028DFDCE0
:10517000019B00982946324607B0F0BD03460B4319
:105180009B0703D009E008C9121F08C0042AFAD2FD
:1051900003E00B780370401C491C521EF9D2704783
:1051A000D2B201E00270401C491EFBD270470022BF
:1051B000F6E710B513460A4604461946FFF7F0FF16
:1051C000204610BD30B504460020034600E05B1CBD
:1051D000934203D2E05CCD5C401BF8D030BDF8B503
:1051E00002464A40D40F42004B0052085B089A42E4
:1051F00002D20246084611464A0023D0C30D4A0097
:10520000DDB2120EAD1A202D35DA49020126490A07
:10521000F6058A19002C00D0524220214F1B11465E
:10522000B9402A411018C20D9A4221D0002C17D043
:10523000012D08DCDA05801AD20F8019D207DBB203
:1052400000F0F6FAF8BDDA05801A012340001B06CB
:10525000C01880185A428018CA0F1043490007E04E
:105260004908C2071143DA05801A801940088018DE
:1052700000F0D6FAF8BD61000122511A001BF7E7D1
:105280000122D2075140AAE70122D2075040A6E7E7
:1052900070B502464A40D50F40004A00ED0740086D
:1052A0005208002814D0002A12D0C40DD30D410298
:1052B0000120C0055202490A520AE41A09181218BC
:1052C0007D34914201D3641C00E04900002C01DAD6
:1052D000002070BD0023914201D3891A0343400886
:1052E00049000028F7D100290AD0914202D10121BA
:1052F000C90705E0914201D2012101E00121C94322
:10530000E005C018401900F08BFA70BDF0B50746F3
:105310000846584087B0C00F049048000E46590018
:1053200040084908BC1A884105D2384631461E4615
:1053300017460B4602465800400810434CD0300D2B
:10534000039040055900400D490D0590401A029008
:10535000402872DA18030121000B09050843019067
:1053600004980092002805D00199524200208841FB
:1053700000920190029840210A1A0199009800F0C9
:105380001BFA05460C466B4607CB00F036FAC019EF
:105390007141039A0E0D0023D71756401A467A40E2
:1053A000164344D0049A002A2DD0029A012A039A67
:1053B00015DC1205C01A914101263605001C714109
:1053C000D20F059ED2070093019202962A462346E9
:1053D00000F074FA07B0F0BD38463146FAE716051A
:1053E000224A0F46B218C01AB74101210905001C14
:1053F0004F4100187F41114618187941E20F1043C0
:105400006D19644113E0E2076D0815436408C20793
:105410001443039A01261205C01A91413605001C57
:105420007141CE07400830434908C01851412A460F
:10543000234600F036FACDE7FFE70498012240004A
:10544000C117121A00238B4104983146C417381A29
:10545000A141EEE730B40124E407634030BC55E7D6
:1054600030B40124E407614030BC4FE70000E0FFA6
:10547000F0B51FB488B00B990998002448400999E9
:10548000C00F490049080991C0070B9900904900D5
:1054900049080B9109990898A64608431CD00B9916
:1054A0000A98084318D0099801244000420D48008A
:1054B000410D099824050003000B204309900B9827
:1054C0000003000B20430B9050181C494018002289
:1054D00001901446104605E0002001460DB0F0BDD5
:1054E000032801DA034600E003239C46C11A0AAEF2
:1054F0000AE05F0008ADED5B4F00F75B7D430027DE
:10550000AA187C41491C5B1E6145F2DD410004ABD9
:105510005A522104120C0A43240C401C0828DFDBD9
:10552000019802900099704601910090059B049AA1
:105530000799069800F0C2F9D0E700000DFCFFFFC4
:10554000F0B50C465C4085B0E40FE40703944C00D2
:1055500000266408590094464908024602962243F0
:1055600021D062460A431ED06200570D4A000E0346
:105570002303550D012402462C492405781B1B0BDF
:10558000360B401823432643614600901C46501AB0
:10559000B44103D30098401C009002E09218009898
:1055A0005B41002803DA0020014605B0F0BD002071
:1055B000012109050746864611E064461D46141B75
:1055C000B54106D36546521BB341744607430C43AD
:1055D000A646CD0740084908284392185B41054676
:1055E0000D43EAD11046184313D060461946504087
:1055F0007140084306D06046101AB34106D201221A
:10560000002306E000220123DB0702E00122D2434F
:105610005310009874460105381C6141029C039D9B
:105620000019694100F03DF9BFE70000FD030000EB
:10563000C217C10F504010B54018CA079623002169
:1056400000F0F6F810BD10B500229623114600F0C8
:10565000EFF810BD0EB5C217C10F5040CA07401871
:105660000021054B0293019200910A460B4600F07F
:1056700025F903B000BD0000330400000EB5054954
:105680000291002100910A460B46019100F016F9A3
:1056900003B000BD33040000410040020122400A73
:1056A000D205090E80187F2901DA0020704796295B
:1056B00003DC9622511AC8407047963988407047DB
:1056C00070B5CD0F4A0009030123090B1B051943CF
:1056D0000B4BED070024520D9A4201DA002070BDF9
:1056E000074B34339A4203DC9A1A00F075F802E053
:1056F0000449511888402C43F1D0404270BD00004D
:10570000FF030000CDFBFFFF4A0009030123090B43
:105710001B051943094B10B5520D9A4201DA0020BE
:1057200010BD064B34339A4203DC9A1A00F054F849
:1057300010BD03495118884010BD0000FF03000050
:10574000CDFBFFFFC20FD207400040080BD0C10DB8
:105750000723DB01C91840020905400A1143C208AA
:10576000400711437047002001467047CB0FDB070D
:10577000490010B5490802460A4307D00A0D07241C
:105780000903E401090B121B002A01DC002010BDF3
:10579000C900440F0C43C100E018D205801800F086
:1057A0003FF810BD0122D207002800DB101A0029A3
:1057B00000DB511A8142704710B5202A04DB0146F4
:1057C000203A9140002010BD914020239C1A0346AE
:1057D000E3401943904010BD10B5202A04DB084671
:1057E000203AD040002110BD0B46D340D0402024A9
:1057F000A21A91400843194610BD10B5202A06DBB5
:10580000CB170846203A1041C1170B4306E00B4660
:105810001341D0402024A21A91400843194610BDDC
:10582000002904DA401C490001D1400840007047BB
:1058300070B40024050C05D11024000402D1002905
:1058400021D01124050E01D100020834050F01D129
:105850000001241D850F01D18000A41C002801DB5C
:105860004000641C002908D020252E1B0D46F54061
:10587000A14000D001212943084301061B1B000A57
:10588000DB1D02D5002070BC7047DB05181880189E
:105890000029F8DA401C4900F5D170BC40084000EE
:1058A000704710B5002B08DA0024401C61419218A3
:1058B0005B411A4301D14008400010BDF0B51FB450
:1058C00082B005460C0003D0084604F087F802E0D9
:1058D00004F084F820300246009021462846FFF765
:1058E0006BFF049B059A04460F4618431143084377
:1058F00014D0184610431BD0009840210A1A1846AD
:105900000599FFF769FF05460E46009A0599049828
:10591000FFF752FF084305D0012004E02046394636
:1059200007B0F0BD0020C11705430E432C43374399
:1059300000990E986305401A7905E40A00220C4389
:10594000FD0A0A3002D500200146E9E701051019D9
:1059500069410C9C0D9D00196941FFF7A2FFDFE72B
:1059600010B5002904DB0124E40740428C412146A4
:10597000002B04DB1C460123DB075242A341994262
:1059800000D1904210BD0000064C0125064E05E0F6
:10599000E36807CC2B430C3C98471034B442F7D350
:1059A000FFF792FBD0A90008F0A9000838B504461B
:1059B000064805490068FFF79BFB604300E0401E76
:1059C00000900028FBD138BD40420F0004010020A8
:1059D000F8B50446006881688907890F012902D15A
:1059E0000168C90722D18168114A1026114001259A
:1059F00000290ED18168294381600120FFF7D6FF7D
:105A000000F0AAFF07460CE000F0A6FFC01B0A2822
:105A100007D9606D30436065A06D2843A065012003
:105A2000F8BD20680068C043C007EDD10020F8BD74
:105A30001700008010B500231A4603E0845CE318C9
:105A40009BB2521C8A42F9D3D84380B210BD0000E9
:105A500010B5034800F040FD024800F03DFD10BDC8
:105A6000F0150020A815002030B5446C1C252C40F2
:105A70000125A540046C6560046863608368102B91
:105A8000036803D099600068C26030BD9A60006806
:105A9000C16030BD1449012048720A4602205E32BE
:105AA000507203203C3A507204200E3A50720F4854
:105AB0000D4B0078087022310870203108770C49AE
:105AC0005A1C0878587149789971233318715971A3
:105AD000203318775977107551751A461E32107594
:105AE000517510765176704738110020C70000209C
:105AF000E400002010B503F037FA202003F0DCFAB0
:105B0000012004F01BFB002003F0D6FA044804F047
:105B1000B9F9044804F05CFC002004F091FC10BDCD
:105B2000B00000208380000070B50520012100072F
:105B300000F002FF00240D4D002800D02C6002214F
:105B40000B4800F0F9FE002808D10A482C600088B4
:105B50000A2148430849088003F092FE012000F022
:105B600023FE022000F020FE70BD0000FC0000209B
:105B700000040050D4000020E00000207047000026
:105B800010B5084900224A6107494B684C15234368
:105B90004B604B68082423434B60C009C00102607E
:105BA00010BD000038160020002002407FB50025FF
:105BB0000C460646039500F0C7FDE009029003A9D4
:105BC00001960095684600F057FD002804D000F0CB
:105BD0008FFD002004B070BD00F08AFD0120F9E7C0
:105BE00010B5002302E0C45CCC545B1C9342FAD392
:105BF00010BD000010B5214A00219069C30520485E
:105C000004D54169022319434161911593699B05AC
:105C100005D5436901242343436163021943936912
:105C20005B0505D54369082423434361E301194318
:105C300093691B0505D5436904242343436163022B
:105C4000194393699B0405D5436910242343436199
:105C50006302194393699B0304D5446920231C43C1
:105C6000446119439369DB0305D543694024234309
:105C70004361A0020143916110BD00000020024079
:105C80003816002070B5054600F066FE0646184C32
:105C90000AE0681C08D0002D04D000F05DFE801BD7
:105CA000A84201D9032070BDA069C007F1D1A06945
:105CB000800701D50220A061A069C00511D4A069A8
:105CC00080050ED4A06940050BD4A069000508D456
:105CD000A069800405D4A069800302D4A069C00330
:105CE00003D5FFF787FF012070BD002070BD0000C5
:105CF00000200240F8B51746002605460C4600F085
:105D000023FD09E029460220226800F0FFFC00285C
:105D100004D1241D2D1D361DBE42F3D300F0E8FC36
:105D2000BE4201D20020F8BD0120F8BD10B50849DF
:105D300002460020054B497905E044001C5B944273
:105D400003D0401CC0B28842F7D310BD60120020BF
:105D50004800002010B500F0F4FD10BD10B5094852
:105D600000F0A0FF80B2FFF789FC074A074BFFF75E
:105D70007FFB0022064BFFF7E3FBFFF7C5FC80B279
:105D800010BD0000A0140020F853E3A59B843E4002
:105D900000408F40F8B540493E488A7F0275C97F70
:105DA00041753E490A78027649784176394905209D
:105DB000133148720A2004F0FBFA7D20C00004F081
:105DC00011FB3449002213310C2004F0DBFB0021CD
:105DD0000C2004F0E9FB022004F03AFB304D2E4C7D
:105DE00000210F2004F064FA28422063F8D0206BD1
:105DF000411C40D02B4E2C4F40043ED58122D20175
:105E000000210F2004F093FB0021102004F050FA31
:105E100041062048490E0022633004F07FFA1D4DF0
:105E20006335687A052825D102221C49681DFFF7D1
:105E3000C9F900281ED1A87C607117480422691C8A
:105E40004430FFF79BF9606C00F034F8A083607970
:105E500029464200133108465130FFF78FF91348A5
:105E600031888088FFF744F9388841431048018021
:105E700003202070F8BD02F01FFAA08B3188054680
:105E8000FFF736F93888414309486D1E0180A58324
:105E9000F8BD00009911002048000020E400002017
:105EA00000D02724D0000020CE000020380D002094
:105EB000CC00002010B504460E4800F0F3FE0E4959
:105EC000C006C00E098805E02246C240D2070FD0A6
:105ED000401CC0B28842F7D3012005E02246C240F0
:105EE000D20705D0401CC0B28842F7D3491EC8B2C1
:105EF00010BD0000A0140020D000002010B50848FC
:105F000000F096FA0A21064800F032FA044800F040
:105F10001DF9800503D5024800F01AF980B210BDC2
:105F200044140020F8B52F4D00220121284600F02E
:105F30000CFDFFF7E3FFFFF786FB2B4E3146FFF723
:105F4000A7F92A4C0122A0601146284600F0FDFC6A
:105F50002749A068002588423EDB2078254F00288D
:105F600015D02570FFF7CAFFFFF76DFB3146FFF72D
:105F70008FF9A060FFF7E6FB00223B46FFF76AFAC5
:105F800000221D4BFFF774FAFFF7F0FB6060A0687A
:105F9000FFF7D8FB00223B46FFF75CFA174A184B85
:105FA000FFF766FA06460F466068FFF7CBFB134A19
:105FB000144B5242FFF75CFA32463B46FFF7A6F914
:105FC000FFF7D4FB10496060884201DD616004E0A6
:105FD000FF21C905C84200D365606068FFF75CFB1C
:105FE000C0B2F8BD0004005000401B442400002053
:105FF0000000604000000C4000E064403333333365
:1060000033B33040CCCCEC3F0000C842F8B5054675
:1060100004464035287C0026012808D00120287439
:10602000206881688907890F01290ED101E00220CB
:10603000F8BD0168C90708D0606D2021084360657C
:106040000126002028743046F8BD616DFF22013220
:106050009143022211436165C1688907890F00914C
:10606000C16889088900C16020688168920711436E
:10607000816000F071FC07460EE000F06DFCC01B73
:106080000A2809D9606D0221884310210843606500
:10609000002028740120F8BD206880680028ECDB0F
:1060A0002068C168009A1143C160606D800880005B
:1060B000401C6065C5E70000F8B506460D46403651
:1060C000317C01290DD00121317401688A685207A1
:1060D00009D5416D20221143416500203074012013
:1060E000F8BD0220F8BD174B6A68D80547109A42E0
:1060F000154C8A6A2B6812D05B035B0B1A438A62C9
:106100002968490305D5A1680143A1600A20FFF76A
:106110004DFC2868800312D5A06838430EE05B036D
:106120005B0B9A438A622968490302D5A1688143BF
:10613000A1602868800302D5A068B843A060002051
:106140003074F8BD0110000000270140406D704719
:106150000068006C7047000070B5040006D0606DE8
:10616000264600254036002802D006E0012070BDFA
:10617000A5653574204600F0D3F8606DC00603D4E1
:1061800021688868400705D5606D10210843606567
:106190003574EBE7606DFF22013290430222104319
:1061A000606588688207920F5B48012A02D10A68FD
:1061B000D2072BD1032362689B079A4205D05B422A
:1061C0009A4202D05B009A4209D10A699200920871
:1061D0000A6121680A6963681A430A610CE00A6966
:1061E000920092080A6181680F22920491438160B3
:1061F00081686268114381602168CA6818239A43E4
:10620000CA602168CA68A3681A43CA60816801220B
:106210005206914381608168A28E520611438160CB
:1062200020688168C90004D48168012212071143E3
:1062300081602068C168394A1140C1602069E16805
:10624000022825D000200143204620300278037B1D
:1062500052035B001A431143226B1143A26992035C
:106260001143E269D20311432268D3681943D16014
:10627000616A0A46FF3AC23A05D0A26A114322680F
:10628000D3681943D16042780121012A02D00BE082
:106290000420D8E70078002823D0606D2022104326
:1062A0006065A06D0843A065E06B012820681FD0E1
:1062B0000169C90703D001694908490001612068E3
:1062C0004169C908C900416120684169A26B114355
:1062D0004161A565606D80088000401C60650020FC
:1062E00070BD2068C26801231B041A43C260DBE74B
:1062F0000269FF239B009A43026120680269236CB4
:10630000A66C1A43636C33431A4302612068026926
:106310000A430261D3E70000002701401902FEFF93
:1063200010B586B0044614216846FEF740FF0E49BA
:106330002068884216D10D48416B421511434163D4
:10634000C16A01221143C162C06A694610400590CA
:1063500002200090032001900020029005200007F9
:1063600000F02EFA06B010BD0024014000100240DB
:10637000F8B504464069254640350E4608280BD03E
:106380002068C068C00709D0606D2021084360659F
:10639000002028740120F8BD082700E00C2700F039
:1063A000DBFA009011E0701C0FD0002E05D000F039
:1063B000D3FA0099401AB04207D9606D042108430E
:1063C0006065002028740320F8BD2068006838420A
:1063D000E9D0606D01214902084360652068C16809
:1063E00009058A0F0C21002A1BD12022125D002AE8
:1063F00017D10268120714D5826853070122002BB7
:1064000008DB43688B434360606D1302984310437D
:10641000606506E0606D202318436065A06D104341
:10642000A065A069002801D1206801600020F8BDA6
:1064300070B50446216800208968490721D42546A3
:106440004035297C01291CD001212974E1690129E9
:1064500004D02046FFF7BCFA002811D1616D0A4A2A
:106460001140FF220132114361650021A1652974A9
:1064700022681C21116021688A6804231A438A60FB
:1064800070BD022070BD0000FEF1FFFF70B500245A
:10649000014620314A79022A03D00421C163012434
:1064A00018E0026813680E25AB4313600268136896
:1064B0005B085B001360436C1C22134001221546ED
:1064C0009D40036C5D604A7100220A71816B002956
:1064D00000D08847204670BDF0B4016C0D6801689B
:1064E0000C68466C1C2304221E401746B7402F42FE
:1064F0000ED067070CD50C68A40602D40C68944330
:106500000C60416C19408A40016C4A60016B1AE0D2
:106510000227B74002462F402032002F17D0A7078E
:1065200015D50C68A40605D40C680A25AC430C608C
:1065300001215171446C02211C40036CA14059603F
:1065400000211171C16A002918D0F0BC0847082742
:10655000B7402F4212D0240710D50C680E25AC434B
:106560000C60446C01211C400B46A340046C63602A
:10657000C163517100211171416BE4E7F0BC7047B8
:1065800070B504003CD01F48256814212818FEF778
:10659000AFFD800060641C4820640221204620304A
:1065A0000246417129681948E3680140A06866699C
:1065B0001843236933431843A3691843E369184315
:1065C000236A1843084328600121A0688903884290
:1065D00010D00D488030836A656C1C210D400F2659
:1065E000AE40B3438362656C63680D40816AAB4023
:1065F0000B4383620020E06301215171107170BD73
:10660000012070BDF8FFFDBF000002400F80FFFFBA
:10661000F8B504468C46203001790025012909D0BF
:106620000126067141790027012905D0077102254D
:106630002846F8BD0220F8BD02214171E7632068B9
:10664000016849084900016061462046FFF70CFADD
:10665000206B00282068016801D00E2205E004228A
:1066600091430160206801680A221143016020689B
:10667000016831430160DBE7F8B51A4E0546307C0E
:106680000F46012807D0012030741748FFF7FAFAA7
:10669000010002D021E00220F8BD0020C043386094
:1066A0006C6814E02046FFF76BFA0F48FFF7EAFA30
:1066B00001460E48426808239A43426042684315E7
:1066C0009A434260002901D03C6006E08034A8680B
:1066D0006A68C0018018A042E4D8002030740846DF
:1066E000F8BD00003816002050C300000020024012
:1066F000054841680222114341604168012211436B
:10670000416000207047000000200240F8B50C4CAA
:106710001646207C0F46012808D001202074094825
:10672000FFF7B0FA0025002802D006E00220F8BDED
:1067300065613E600348FFF7A5FA2574F8BD0000C7
:106740003816002050C3000011484168C9070BD01B
:10675000EFF3108172B60F4AC2600F4AC26081F334
:1067600010884168C9070ED1416889070DD5EFF33C
:10677000108172B6094A0261094A026181F31088E8
:106780004068800701D50120704700207047000055
:1067900000200240EFCDAB8905040302BFAE9D8C03
:1067A000161514137047000010B504494A690242D7
:1067B00002D04861FFF7F6FF10BD00000004014061
:1067C000F8B500230124A2E027469F403A4070D04C
:1067D0004D68022D01D0122D14D1DD08AD002D1809
:1067E00000952D6A5E07AC46F50E0F26AE46AE400C
:1067F0006546B543AC460E697546AE4065462E43C8
:10680000009D2E624D68012D05D0022D03D0112D63
:1068100001D0122D16D185680326AC465D00AE4628
:10682000AE406546B543AC46CE687546AE4065465B
:106830002E43866046680D79BE43ED06ED0F9D4000
:106840003543456006685F000325BD40AE46AE4354
:106850000D79B446AE07B60FBE4065462E430660BE
:10686000C6687546AE438D68BD403543C5604D680A
:10687000ED004BD5294D6E6B26436E639E08284D67
:10688000B6007519AC46AD689E07360F0F27B740A6
:10689000BD4305273F07B84201D1002715E0214F2E
:1068A000B84201D1012710E01F4FB84202D10227A0
:1068B0000BE02BE01D4FB84201D1032705E01C4F30
:1068C000B84201D1052700E00627B7402F436546AF
:1068D000AF60184D2E684F689643FF0300D51643EE
:1068E0002E606E684F689643BF0300D516436E60F6
:1068F000AE684F689643FF0200D51643AE60EE685F
:106900004F689643BF0200D51643EE605B1C0A68D1
:106910001546DD4000D057E7F8BD000000100240EA
:10692000000001400004005000080050000C00501E
:10693000001C0050000401400069084000D0012004
:10694000704742694A4042617047002A01D0816124
:10695000704781627047000001480068704700007E
:106960000001002002480168491C016070470000D6
:106970000001002010B5084800240168402211439E
:106980000160204600F00AF8002801D0012401E04F
:1069900000F0B4F9204610BD0020024070B5054655
:1069A00009487D210024C9000068FEF7A1FB00F022
:1069B00049FE002801D0012404E000222946501E8F
:1069C00000F0BCF9204670BD0401002070477047FC
:1069D000F8B52D4C0126A078401CA0702671E08AE5
:1069E000401CE0822948008802F024FB284DE888FA
:1069F000FEF729FE2749FEF74BFC274F3968FEF7C3
:106A0000EEFB386002212548FFF796FF002700289B
:106A100009D027632048224A016822480091914208
:106A200012DD067011E0E888FEF70DFE1949FEF749
:106A30002FFC216BFEF7D3FB1B4920638842E9DB67
:106A40001B491A48C860E5E70770688F401EFEF7CB
:106A5000EFFD0099FEF7A6FE05D86079002802D068
:106A60001448067001E013480770688FFEF7EBFDCD
:106A700009490968FEF796FE04D26079002801D022
:106A800003F07AFEF8BD0000C4000020640000207E
:106A9000380D002000007A44FC0000200004005063
:106AA000000040404E0000200000A0400400FA0515
:106AB00000ED00E05D000020704770B505000DD0CE
:106AC00002202C462034A073284601F017FA2846ED
:106AD00000F0BEF80020A073607370BD012070BD8F
:106AE0007047704710B5044600680168C943C9077C
:106AF00008D18168C943C90704D1012141602046FA
:106B0000FFF766FF20680168C943890708D48168D8
:106B1000C943890704D4022141602046FFF756FF8C
:106B200020680168C943490708D48168C9434907F7
:106B300004D404214160204600F0DEF8206801689A
:106B4000C943090708D48168C943090704D4082147
:106B500041602046FFF7B0FF20680168C943C906BD
:106B600008D48168C943C90604D410214160204675
:106B7000FFF72DFF20680168C943890608D48168A2
:106B8000C943890604D4202141602046FFF7A9FFAC
:106B900020680168C943490608D48168C943490689
:106BA00004D4402141602046FFF79AFF10BD000049
:106BB000F8B5040005D025462035A87B002802D072
:106BC00006E00120F8BD00206873204600F052F86E
:106BD0000220A8732068C26884466368012B04D031
:106BE0000120A16AC005814201D11E2082431548BF
:106BF0006169814201D0144802401448A6680240ED
:106C000018463043676A266A3E433043A66A3043DB
:106C10001043012B03D00122D205964203D12369F0
:106C2000E2681A431043074A914205D0A269114312
:106C3000E2690243084610436146C8600120A87318
:106C40000020F8BDFFFF00003F1FFFFFF8F119FF14
:106C500010B500680549884207D10548816B490095
:106C6000490881630D2000F055F810BD007C0040FC
:106C70000010024010B50068084988420CD108484D
:106C8000816BC20411438163002201210D2000F0B9
:106C900055F80D2000F048F810BD0000007C0040C1
:106CA000001002400068C0697047000070B50224FF
:106CB000034620339C730F4C2568E604354325605A
:106CC0000468E568B6123543E5600568AE680124DE
:106CD0002643AE6005682E6926432E610568A961CA
:106CE00001684A61006801690422114301619C73D3
:106CF000002070BD00040140704700000448416B53
:106D0000012211434163816B020411438163704787
:106D100000100240C106C90E0120884001490860E8
:106D20007047000080E100E0C106C90E01208840E4
:106D3000014908607047000000E100E010B501F073
:106D400099FA10BD02494A6882434A6070470000C0
:106D500000700040024801688215114301607047CD
:106D60000070004002494A6802434A6070470000D0
:106D70000070004005480168022211430160044888
:106D8000016904221143016130BF70470070004067
:106D900000ED00E00A4B1A689208920002431A6064
:106DA00008480369042213430361012906D040BF48
:106DB00020BF20BF016991430161704730BFF9E7EF
:106DC0000070004000ED00E0F8B504460078544D36
:106DD000800672D5524E0027403EB06BC00004D4EE
:106DE000B06BA9050843B06301274E480168C90587
:106DF00011D40168821511430160FFF7ADFD0090C9
:106E000005E0FFF7A9FD0099401A642837D84548E6
:106E10000068C005F5D532680321090560680A409D
:106E20000140914208D08103890F032904D13168C0
:106E3000890301D50120F8BD2A69032109040A400C
:106E400022D0084090421FD0207880061CD52869A7
:106E50002A6988430121C9040A432A612A698A43AD
:106E60002A612861C0050FD5FFF776FD009008E084
:106E7000FFF772FD0099411A2B48814201D9032086
:106E8000F8BD28698005F3D561688803800F032861
:106E900005D132680005824301400A433260286907
:106EA000032261681204114008432861002F04D0B6
:106EB000B16B012000078143B1632078C00705D082
:106EC000E868A168800880000843E86020788007AF
:106ED00005D5E8680C218843E1680843E86020781C
:106EE000400706D5E86803218902884321690843E1
:106EF000E8602078000706D5E86803210903884385
:106F000061690843E8602078000606D5E868032137
:106F100089048843A1690843E8600020F8BD0000A7
:106F2000401002400070004088130000F8B50E4683
:106F300005007DD053480068C007C00FB0420AD298
:106F40005048016849084900314301600068C007A2
:106F5000C00FB04271D128784B4C800705D5E0684E
:106F6000F0218843A9680843E0602878C00752D020
:106F70006868022817D0032818D02168012818D083
:106F80008905002959DAE168890889000143E1602F
:106F9000FFF7E2FC69680746022912D003291CD0DA
:106FA000012926D033E021688903EAE721688901B5
:106FB000E7E74907E5E7FFF7CFFCC11B334881420C
:106FC00023D8E0680007800F0228F4D123E0FFF700
:106FD000C3FCC11B2D48814217D8E0680007800F11
:106FE0000328F4D117E0FFF7B7FCC11B2748814203
:106FF0000BD8E0680007800F0128F4D10BE0FFF701
:10700000ABFCC11B2148814201D90320F8BDE068D7
:107010000007800FF3D11B480168C907C90FB142AF
:107020000DD901684908490031430160006800E05A
:1070300003E0C007C00FB04201D00120F8BD28789E
:10704000400706D5E068072109028843E96808433C
:10705000E0602878000707D5E0680721C902884367
:107060002969C9000843E06000F036F8E168084A81
:107070000906090F515CC840064908600020FFF767
:107080008DFCF8BD00200240001002408813000073
:10709000AEA9000804010020044805490068C96839
:1070A000044A4905490F515CC8407047040100205B
:1070B00000100240C7A90008044805490068C968D3
:1070C000044A8904490F515CC840704704010020FC
:1070D00000100240C7A9000810B5184AD1680C205A
:1070E000084004280BD0082810D00C2810D0506875
:1070F0000004410F0120C003491C884010BD1068E6
:10710000C00601D50E4810BD0E4810BD0E4810BD7A
:1071100088020E4B000F185C0902D368890F491CC6
:10712000DB0301D5084A05E01268D20601D5044AFE
:1071300000E0044A5043FDF7DBFF10BD00100240A1
:1071400000093D000024F40000127A00BEA90008E6
:10715000FEB505007ED0FE4CE7680C20E6680740CF
:107160000120000406402878C00747D0082F05D02A
:107170000C2F0AD101200004864206D1206880032A
:107180003CD568680028E5D038E001206968000433
:10719000814203D121680143216011E005230122CE
:1071A0001B0492049942216802D111432160F1E746
:1071B0008143216021680140009120689043206054
:1071C000686800280DD0FFF7C7FB009005E0FFF7C7
:1071D000C3FB0099401A64287AD820688003F6D54A
:1071E0000CE0FFF7B9FB009005E0FFF7B5FB009955
:1071F000401A6428F0D820688003F6D428788007E5
:1072000055D50923E868042F0DD00C2F01D1002E8D
:1072100009D000283BD02168994301432160FFF742
:107220009BFB064627E02168490701D5002891D03D
:1072300061681F22120291432A69120211436160A0
:107240002168994301432160FFF746FFE168090681
:107250000A0F00E079E1BF49895CC840BE49086077
:107260000020FFF79BFB002872D120E0FFF774FBA2
:10727000801B0228B0D820684007F7D560681F211E
:107280000902884329690902084360600FE0206809
:10729000400840002060FFF75FFB064604E0FFF770
:1072A0005BFB801B022897D820684007F7D428781A
:1072B000C0065FD5002F0CD0A869002849D02068EF
:1072C000FF21013108432060FFF746FB06462DE011
:1072D000C0E02068800502D5A8690028A7D06068B2
:1072E000072149038843296A084360606068297F51
:1072F0000002000A090608436060286A410B012069
:10730000C003491C8840E16809060A0F9149895C5D
:10731000C840914908600020FFF740FB002817D1C2
:1073200028E0FFF719FB801B0228A3D820688005FE
:10733000F7D56068072149038843296A08436060DC
:107340006068297F0002000A09060843606011E0B6
:10735000E1E02168FF20013081432160FFF7FCFA62
:10736000064604E0FFF7F8FA801B022872D820686E
:107370008005F7D42878794E000724D5686900285D
:10738000306910D0012108433061FFF7E5FA009021
:1073900005E0FFF7E1FA0099401A02285AD830694F
:1073A0008007F6D50FE0400840003061FFF7D4FABF
:1073B000009005E0FFF7D0FA0099401A022849D85A
:1073C00030698007F6D42878400765D50020029000
:1073D000A06BC00006D4A06B012109070843A0637D
:1073E000012002905E480168C90511D40168821528
:1073F00011430160FFF7B0FA009005E0FFF7ACFA27
:107400000099401A642825D855480068C005F5D56C
:10741000FF20AA680130824203D131690143316102
:1074200011E001218902002A07D005231B029A429C
:1074300003D132690A433261EFE732698243326134
:10744000306988433061A86800280FD0FFF784FABC
:10745000009007E05EE0FFF77FFA0099411A41488B
:10746000814257D830698005F5D50DE0FFF774FAF1
:10747000009006E0FFF770FA0099411A39488142FE
:1074800048D830698005F5D40298002804D0A06B54
:10749000012109078843A063686A002864D00C2F83
:1074A0003ED0012636060228206805D0B043206071
:1074B000FFF752FA05462FE0B0432060FFF74CFA81
:1074C000074604E0FFF748FAC01B022822D82068CC
:1074D0008001F7D4E96AA86AE2680843296BFD23B2
:1074E0001B049A4311430843E06020683043206046
:1074F000FFF732FA054604E0FFF72EFA401B022898
:1075000008D820688001F7D52EE0FFF725FA401B48
:10751000022801D90320FEBD20688001F5D423E0B4
:107520000128F8D0E06801210904AA6A01409142CB
:107530000BD10F218904EA6A0140914205D1032150
:1075400089050840296B88420ED00120FEBD00004D
:1075500000100240AEA900080401002040100240C3
:1075600000700040881300000020EFE770B50400B1
:1075700007D0002625464035A662687C002802D048
:1075800005E0012070BD2E74204600F02FF8022087
:10759000687420680168402291430160A1686068B6
:1075A00022690843E16811430843616901220843E5
:1075B000A169520211400843E1690843216A084366
:1075C000A16A084321680860A0690421000C0840F2
:1075D000616A0843216848602068C169920091434C
:1075E000C161666501206874002070BD10B586B069
:1075F000044614216846FDF7DAFD104920688842E8
:1076000019D10F48416B821411434163C16A0122B1
:107610001143C162C06A002110400590E020009033
:1076200002200190032003900291049105206946F5
:107630000007FFF7C5F806B010BD0000003001409C
:1076400000100240094910B5401E884201D90120AE
:1076500010BD074C60610321081F00F00BFE0020E5
:10766000A06107202061002010BD0000FFFFFF0087
:1076700000E000E070477047F8B502680446D06942
:107680001168936805072D0F5BD0DD07ED0FFF260E
:1076900021360E402E4367D0C60706D0CE0504D54E
:1076A00001261662E26F3243E26787070222042650
:1076B000002F06DADF0704D027683A62E76F374306
:1076C000E767470706D5DB0704D023681E62E36F30
:1076D0001343E367020709D520220A402A4305D055
:1076E000236808221A62E36F1343E367E26F002AFC
:1076F0002FD0800606D5880604D5216E002901D03A
:1077000020468847E06F21688968490601D4000750
:1077100024D5204601F012FF20688168490619D55A
:107720008168402291438160E06E002812D0204998
:107730008163E06EFEF7AAFE00280AD0E06E816B3E
:1077400006E0850610D58D060ED5216E1CE020467C
:107750008847F8BD2046FFF78EFFF8BD2046FFF7AB
:107760008AFF0020E067F8BDC50208D55B0206D598
:107770000120000510622046FFF77CFFF8BD0306DC
:1077800005D50B0603D5616E0029E0D1F8BD400692
:10779000FCD54806FAD51368204640218B43136078
:1077A000202161670021616600F069F9F8BD0000E1
:1077B0009994000810B5040003D0606F002802D02F
:1077C00007E0012010BD002170200155204600F087
:1077D00027F8242060672068016849084900016093
:1077E000204601F0F5FE0128ECD0606A002802D0A6
:1077F000204601F033FD206841680922D2029143FE
:107800004160206881682A22914381602068016874
:10781000012211430160204601F086FD10BD0000E9
:10782000F0B587B0064614216846FDF7C0FC2C4928
:107830003068884251D12B48416B01229203114399
:107840004163C16A01221143C162C06A0025104030
:1078500005900320400200900220032701A9A1C146
:1078600004200490052069460007FEF7A9FF1F4C7D
:107870001D48A560E56081C48027E560A7602020E1
:10788000256160610002A0611848083CFEF778FE9F
:10789000002801D0FEF772F9F466A662144C124873
:1078A0002146143820600320606010200831A1C1F7
:1078B0006561A561E56120462562FEF761FE00284D
:1078C00001D0FEF75BF9B466002201211B20A662FD
:1078D000FFF734FA1B20FFF727FA07B0F0BD0000CE
:1078E000003801400010024030000240A81500207E
:1078F000F0150020F8B50446806F20284DD10029EE
:107900000BD0002A09D00123A0681B03984206D19E
:107910002069002803D1C80701D00120F8BD254601
:107920006035287C012838D00120287458206165F2
:1079300002530026E6672220A067E06E002819D0D7
:107940001749C162E16E17480863E16E1648486343
:10795000E06E13468663676D21683A462431E06E17
:10796000FEF756FE002805D01020E0672E74202078
:107970006067D2E72E7420680168FF22013211434C
:10798000016020688168012211438160206881685C
:107990004022114381600020F8BD0220F8BD0000A4
:1079A000F594000833950008AD94000870477047BF
:1079B000FFB50446406F83B017460D4620285CD1C2
:1079C000002D0AD0002F08D0A168C001814207D144
:1079D0002069002804D1E80702D0012007B0F0BDDB
:1079E000204660300290007C012846D00298012198
:1079F00001740020E06721206067FEF7ADFF264696
:107A000040360190378277820120A16800038142CD
:107A100002D12069002802D02F46002511E000275E
:107A20000FE000228021204601F0E6FE002815D15B
:107A3000002F15D02168387888627F1C708A401E1C
:107A40007082708A019B002806980090E9D100227C
:107A50004021204601F0D0FE002808D00320BDE7D9
:107A600028882168C005C00D8862AD1CE6E720208B
:107A70006067029900200874B0E70220AEE7704703
:107A800001490248C160FDE70400FA0500ED00E08D
:107A900010B505242407002204212046FEF755FFD7
:107AA000002208212046FEF750FF0A2002F0A3F929
:107AB000012204212046FEF748FF0A2002F09BF92C
:107AC000002204212046FEF740FF10BD10B505241A
:107AD0002407002204212046FEF737FF0122082157
:107AE0002046FEF732FF0A2002F085F90122042128
:107AF0002046FEF72AFF0A2002F07DF90022042129
:107B00002046FEF722FF10BDF8B5002405260746E3
:107B100025463607002204213046FEF716FF0A20CC
:107B200002F069F9012204213046FEF70EFF6006DB
:107B3000040E08213046FEF7FFFE002801D0641C29
:107B4000E4B2052002F057F96D1CEDB2082DE1D327
:107B5000002F03D0FFF79CFF2046F8BDFFF7B6FFCC
:107B6000FAE770B50526054636070022042130469F
:107B7000FEF7EBFE0024E80901D0012200E000221C
:107B800008213046FEF7E1FE6806050E0A2002F0E5
:107B900032F9012204213046FEF7D7FE0A2002F016
:107BA0002AF9002204213046FEF7CFFE0A2002F017
:107BB00022F9641CE4B2082CDDD370BD10B5052495
:107BC0002407012208212046FEF7BFFE01220421DE
:107BD0002046FEF7BAFE002208212046FEF7B5FE39
:107BE0000A2002F008F9002204212046FEF7ADFE2B
:107BF00010BD10B505242407002204212046FEF7FD
:107C0000A4FE002208212046FEF79FFE0A2002F073
:107C1000F2F8012204212046FEF797FE01220821F6
:107C20002046FEF792FE0A2002F0E5F810BD70B57E
:107C300005252D070024012208212846FEF785FE90
:107C4000062002F0D8F8012204212846FEF77DFE26
:107C5000062002F0D0F807E0641CE4B2FA2C03D945
:107C6000FFF7C7FF012070BD08212846FEF764FE1C
:107C70000028F1D1002204212846FEF766FE0020EC
:107C800070BD0000F8B501F07FFB01F0B9FB4C4876
:107C90000068C0694B4E4C4F800700D5FE60FEF770
:107CA0005DF84A4C024660884949002803D0401ECE
:107CB000608001200870087801218902454D002864
:107CC0001CD0012804D0022804D0032806D115E0D6
:107CD000212A13D200222846FEF737FE0121C902CD
:107CE0003C48FEF729FE3C490025002828D03B48A7
:107CF00005600846C079002802D006E00122EAE7C4
:107D000035490120C87101F0BBFD33480078632874
:107D100006D9002208212F48FEF717FE012205E0B0
:107D2000012208212B48FEF710FE00220121052028
:107D3000C9030007FEF709FEA08C012803D01CE050
:107D4000CD710022EDE726486946088072B6802191
:107D50002448FDF72BFF002804D002226946214861
:107D6000FDF7C8FF62B620A001F028FEA58402F04E
:107D70009FFD642002F038F8FE60608C012809D174
:107D8000124865844038058002F092FD642002F0BC
:107D90002BF8FE60208C012806D1258402F088FD96
:107DA000642002F021F8FE600848134A4038018838
:107DB000914202D1C088002800D1FE60F8BD0000C9
:107DC000281500200400FA0500ED00E0780D0020E1
:107DD0005B00002000040050C4000020FC000020D4
:107DE000AAAA0000384A0008BDF8C8EBC9FDBCB615
:107DF000C4A3CABD0D0A0000AA55000008B537216A
:107E0000202000F06EF80321212000F06AF84021C4
:107E1000222000F066F80821232000F062F8AA2151
:107E2000302000F05EF80A4802210187322000F07D
:107E300058F80121332000F054F85F21202000F091
:107E400050F8684600F006F80A2001F0D4FF08BD9B
:107E5000380D002010B501460F2000F021F8002851
:107E600000D0012010BD10B50446FFF7A7FE322058
:107E7000FFF777FEFFF7DBFEE0B2FFF772FEFFF7DA
:107E8000D6FEFFF79BFE3320FFF76BFEFFF7CFFE1A
:107E90000020FFF739FE0446FFF7ABFE204610BD79
:107EA00010B50C46FFF7DFFF2070012010BD70B544
:107EB0000D460446FFF782FE3220FFF752FEFFF721
:107EC000B6FEE0B2FFF74DFEFFF7B1FE2846FFF722
:107ED00048FEFFF7ACFEFFF78CFE0A2001F08BFF97
:107EE00070BD10B5FFF7E3FF012010BD10B50248CB
:107EF000FEF7F8FD10BD0000A0140020FEB50446FA
:107F0000002572B60068394A831804D13849CD6813
:107F1000032189040D4081680191C1680091416984
:107F20008669002B08D132484038836AC7043B4336
:107F30008362836ABB4383620846304348D02B4840
:107F40002368C34205D12A48C3680322920493439D
:107F5000C360002917D02068026901231A43026117
:107F600020684161FEF7F8FC0746FEF7F5FC216842
:107F7000C01B0968090703D47D21C9008842F4D9D0
:107F8000216808204860002E17D02068016901226E
:107F90001143016120688661FEF7DEFC7D270646FD
:107FA000FF00FEF7D9FC2168801B0968C90601D4CF
:107FB000B842F6D92168102048600C482168C142B7
:107FC00006D10B48C1680322920491432943C16042
:107FD00020680169490849000161216801988860A9
:107FE00021680098C86062B6FEBD00000084FFBF33
:107FF000401002401CB5002116480091144A01911E
:108000000260C1631205426081600722826301221F
:1080100002610246C16020321170FF235170C233E9
:108020004362816211730163816104224163426191
:10803000C161FEF791F808480090801301906946ED
:108040000448FEF739F800210248FDF7DFFF1CBDA8
:1080500000240140441400200200000408B5084830
:10806000016B012211430163006B0121104000905C
:1080700000220A20FEF762FE0A20FEF755FE08BD28
:1080800000100240F0B587B014216846FDF78FF864
:108090004C48C26A04210A43C262C26A0A4005927D
:1080A000C16A80273943C162C16A39400591C16AFA
:1080B00001252943C162C16A29400591C16A02268E
:1080C0003143C162C06A2A463040059005201C2118
:1080D0000007FEF73AFC01223B493C48FEF735FC1D
:1080E00000223B493948FEF730FC9121052000224F
:1080F00009020007FEF729FC3648019000240520FC
:108100006946009502940007FEF75AFB0320019090
:1081100005206946009602940007FEF751FB0C20EB
:1081200000901120019003200390052002946946DD
:108130000007FEF745FB10200090052069460396D6
:10814000019502940007FEF73BFB11200190029479
:108150006946009503941D48FEF732FB1E480190C6
:108160006946009602951948FEF72AFB1B480090C5
:1081700002946946019503941448FEF721FBE80236
:108180006A4651C269461148FEF71AFB9120000267
:108190000090052002946946019503940007FEF7BC
:1081A0000FFB69460948009702950194FEF708FB0A
:1081B000002201210520FEF7C1FD0520FEF7B4FDD8
:1081C00007B0F0BD0010024001060000000400509E
:1081D00008300000000011100000211008360000D7
:1081E00010B50F4C0D482060FF2005306060002066
:1081F000A060E06020616061E061012120624902CD
:108200006062A161A0620720E0622046FFF7AEF93C
:108210002068016840221143016010BD0030014018
:10822000D014002000B585B014216846FCF7BFFFCC
:108230000E480D490160E121490241600021816041
:10824000C160016181610C22C16142610162302122
:1082500041620121090381634900C163FFF7AAFA62
:1082600001F008FB05B000BD0038014028150020D2
:10827000704700008307FF22DB0E9A408907090E32
:10828000994000280BDA0007000F083883080848D7
:108290009B001818C36993430B43C361704783085D
:1082A00004489B001B1818689043084318607047E7
:1082B00000ED00E000E400E0BFF34F8F0449034805
:1082C000C860BFF34F8F00BFFDE700000400FA0550
:1082D00000ED00E0F0B58DB00A2002F069F87D20D5
:1082E000C00002F07FF8FF4C0025A570E07B0C2851
:1082F00001D30B20E0730122052051020007FEF795
:1083000024FBE570F848E574F84E007830710221DE
:10831000F748FEF711FB002864D00020A179F34E46
:1083200049000843617D89000843F071E06AF070FC
:10833000401CE06260793146B0744200B4310846B6
:10834000A138FCF71BFF06207072E649304613384F
:108350008A7F0275C97F41756079002240003146ED
:10836000153002F00FF9607900214000153002F05D
:108370001BF9022002F06CF80025F5716574E572B6
:10838000012060732573DB48FEF78CFC6084064691
:10839000E5706079FDF772F9D74AD84BFDF768F8B8
:1083A00001F0BEFC012300229B07FCF7AFFFFDF7A5
:1083B000ABF90006C10C881980B20121C903A08461
:1083C000884201D3401AA084CD48A0632079401C84
:1083D0002071C848FEF766FC2084C448C94D4E3061
:1083E00005905AE1012099E7C248FEF75BFC208422
:1083F000C54F26460AE0BF48FEF754FC80B23084E1
:10840000B18C884202D34919884206D300210F203B
:1084100001F04EFF38423063EDD0306B411C20D06C
:1084200040047DD58122D20100210F2002F07FF887
:108430007D20C00001F0D6FF002001F088FF002160
:10844000102001F035FF4106A848490E00225030A7
:10845000B16401F063FFA5485030417A0729C0D1CB
:1084600001E0FFF729FFA1480222A8495530FCF797
:10847000A9FE0028B5D102F0E8F87165306502F078
:10848000D1F8F165B065F0786946401CF070974806
:108490004D3002790A70407948700888F18B884223
:1084A0007ED105989A4F008A388090488D494C308B
:1084B000808A48838F48FEF7F5FB3084708B95499E
:1084C000FF30C33080B2708388420CD949424018D3
:1084D000708338888F49401C80B20B3138808842C5
:1084E00001D30020388005987E4A81899186C08911
:1084F000D086726BB2637D4A5032D37C1A07120F5A
:10850000032A00D0F2741A09327500233371012353
:10851000F372744B002A1987588715D0022200E0A5
:10852000AFE0724879495530FCF74CFE00280BD17A
:1085300001206E497074C871B06C64311638C2B2D3
:10854000B2747548FCF71AFE01203073674965481C
:10855000042251314430FCF711FE6448F36D1630AB
:10856000B26D02F047F838887D21C900728B414313
:108570008918F163079169490988CAB23274521E99
:10858000914201D101213173F0841620305EFDF754
:1085900061F800910490308CFDF770F8604A00E0BB
:1085A00013E0604BFCF764FF074603910798FDF763
:1085B00051F83A46039BFCF74DFF009B049AFCF7E9
:1085C000A5FEFDF77DF8306467E0FDF7AFFB0746D9
:1085D000514803210C38C1550598424982898A8641
:1085E000C089C8864C4AB8009C3A716B11503F490B
:1085F000F36D40181A30B26D01F0FCFF70797F1CEA
:1086000087424AD101F072FDFF23A26D5B04E06D49
:108610000021D21848410006150A0543690849009F
:10862000080E0902216660663048636D0A30226DCB
:1086300001F0E0FF2D48636E1230226E01F0DAFF88
:108640002A480821417260790022800027491C30A5
:1086500001F098FF6079002180001C3001F0A4FF38
:10866000284601F09EFE012001F0F2FE0006000EF9
:1086700060721AD100210F2001F01AFE0006F9D510
:1086800013E03A4600210F2001F051FFF178707994
:10869000814202D0002001F05AFE218CA08C814240
:1086A00000D2A1E640198142FBD8174A00210F20D1
:1086B00001F03DFF0021E17363790846049341E036
:1086C000154D0C3D2A5C002A3AD0E67B8F00761CC3
:1086D000E673303DEA51BC464600903DAE5B4F002C
:1086E000183521E048000020C4000020AC11002013
:1086F00000040050A0140020B81E85EB51B8CE3FF6
:10870000A0860100983A000000D02724E400002051
:10871000F8000020E70300002C130020DA000020FE
:10872000F853E3A59B843E40EE5386001835AE59BE
:1087300067463035EE51491C6035521EC9B22A5485
:10874000401CC0B29842BBD3E078032801D2E07B42
:10875000E0734B490022C87B8873401E31E0002142
:108760002BE0484C8B001E19B446E5587668B5429C
:1087700021DD0695434D4C00483D2F5B7835BE46C4
:108780009700ED5905953F4D7746EE50483D6519E8
:108790003C4E0B956D88483E3553344678341E194F
:1087A000384D74683035EC506346069D5D600B9D16
:1087B0006F80059D7560491CC9B28142D1DB521C96
:1087C000D2B28242CBDB2F4802682D48816B32390E
:1087D0008A421BDA2B4930310968002916D0C17949
:1087E000491CCAB2C271032A05D9264948390A88E8
:1087F000C283022202700179032901D9012101708B
:10880000204C00210278603C049B09E00021C171EA
:10881000F1E74D00655B002D00D10222491CC9B271
:108820009942F6D30270174B0021174A303B8C0057
:10883000491CC9B21A510C29F9D3407C002806D032
:1088400010496C3108784B788A7802280DD00F4A8D
:1088500000210F2001F06BFE0121052000224902BA
:108860000007FEF772F80DB0F0BD0948C91CC0182A
:10887000FCF784FC02F01CF8642001F0B5FAF0E586
:1088800048000020C0120020FFFF010080D02724F4
:10889000380D002070470000F0B58DB0B54801904C
:1088A0000020C0430A9000260A2001F081FD7D20AF
:1088B000C00001F097FD0020AF4C0546A070AF4FFF
:1088C000AF480B90AE480022C23885730146142091
:1088D00001F058FE0021142001F066FE022001F094
:1088E000B7FD00210F2001F0E3FC38422063F8D0EF
:1088F000206B411C18D040047ED58122D20100217A
:108900000F2001F014FE0021102001F0D1FC4106DF
:108910009B48490E0022801C01F000FD9848801CF5
:10892000417A022902D005E1FFF7C6FC94480222F1
:108930009449C01DFCF746FC0028F4D101F085FEE7
:108940006165206501F06EFEE165A065002E23D112
:108950000B988D49008A088089488749801E808A43
:10896000488301268948FEF79DF92084608B884959
:10897000FF30C33080B2608388420DD9494240182D
:10898000814960830888824A401C80B20B3208808B
:10899000904201D3002008800B9968468A890280A2
:1089A000C989418076490422C91C0846A238FCF7CF
:1089B000E5FBFF22A16D5204E06D002389185841A8
:1089C0000006090A01430846029101F0EAFC0299F7
:1089D00048084000010E0002616620666848636D29
:1089E0009638226D01F006FE6548E36D9238A26D5F
:1089F00001F000FE624800E09EE08E38636E226E59
:108A000001F0F8FD5E490022A0393C2001F0BAFDDA
:108A100000213C2001F0C8FD012001F019FD607229
:108A2000A0780121401CA0700520C9030007FDF7B4
:108A300091F955487D220088D200014602905043AA
:108A4000628B0A398018E0630C90524800782074D9
:108A5000049008B22085002803DA7D21C90040185F
:108A600020854D48302100884843FCF7ECFD0590F7
:108A70002820205EFCF7DCFD0599FCF709FC7F212E
:108A8000C905FCF7ACFBFCF707FE424980B2088041
:108A90000499491E884201D1012020730298E08484
:108AA0001620205EFCF7D6FD05910690208CFCF781
:108AB000E5FD3A4A3A4BFCF7DBFC079104900C9831
:108AC000FCF7C8FD079B049AFCF7C4FC059B069ABB
:108AD000FCF71CFCFCF7F4FD2064A08B00F0AAFA64
:108AE0000099019881420DDA00290BD02449042213
:108AF000C91C0AA8FCF742FB022020700520A072C6
:108B000000980190607A002805D100210F2001F023
:108B1000CFFB0006F9D5802200210F2001F007FDD0
:108B200000206D1CEDB26070032D00D2CAE6002E4D
:108B300008D01AE00120F4E71A4A00210F2001F0C2
:108B4000F6FCF7E7A08B1849401E0004000CA08338
:108B500002D00A88904201D90888A0831349A08BCB
:108B60000988401E4843124908800A98E0830DB0E6
:108B7000F0BD00003F420F004800002000D0272435
:108B8000FA110020E4000020F8000020A0140020CA
:108B9000E7030000DA000020DE000020F853E3A520
:108BA0009B843E4000902724D0000020CE0000206F
:108BB000CC000020F8B52F492D48086001F018FEC0
:108BC0002E4D2D486880E888002801D16420E88077
:108BD0002B4801783C2901D93C210170E98E0170B4
:108BE000284CE88F6071A88FA071A87AE070AE88D9
:108BF000052126626181EF883846FCF779FAA08169
:108C000001463046FCF774FA8800081886B27D20C9
:108C1000C00026817043FCF731FD1B4A1B4BFCF75B
:108C20008FFCFCF771FDE0817D2066823946C00033
:108C3000FCF75EFA20820146C820FCF759FA6083EF
:108C40000120E082FDF78AF8A082E28910491148EC
:108C5000FEF72CF810A0216A00F0B0FEE98812A0FF
:108C600000F0ACFE298915A000F0A8FEF8BD0000B8
:108C7000AD9800084400002005020000380D0020D7
:108C800000000020C4000020F853E3A59B843E4070
:108C9000FF7F0000A0140020B1EAC7A949443A2090
:108CA0002564202E0D0A0000CDA8D1B6BCE4B8F48E
:108CB0003A202564206D732E0D0A0000B5A5B4CEB0
:108CC000CDA8D1B6BBF9D5BECAFDC1BF3A20256437
:108CD000B8F62E0D0A000000F0B5924D85B00120C7
:108CE0002880914FC820914C3880207A401C2072F7
:108CF000C00706D0A08B411EA183022801D2C82044
:108D0000A083A08B00F096F90A2001F051FB7D2092
:108D1000C00001F067FB02218548FDF70DFE002829
:108D200038D00020834980000978844E49000843E8
:108D3000814909780843B072102070728048C18858
:108D40007D20C000FCF7D4F970737E487C49007820
:108D5000B07330460B308A780270C9784170411C7C
:108D600077482030027ECA70407E087174482230F5
:108D7000027E4A71407E887100220C39152001F074
:108D800001FC0021152001F00FFC022001F060FB26
:108D90006D4E03E00120C5E7FEF774FF00210F20B0
:108DA00001F086FA30422063F6D0206B411C7DD062
:108DB00040047CD58122D20100210F2001F0B7FBB5
:108DC0000021102001F074FA41065C48490E00228F
:108DD0005030A16401F0A2FA584E5036707A112832
:108DE00065D102225949701DFCF7ECF900285ED1CB
:108DF000F01E027969460A7040794870B17A29807C
:108E0000C820FCF775F93880307BA083504DB01E28
:108E1000008A28804549301F808A48834D48FDF7E5
:108E200041FF80B220840390608B4B49FF30C330F8
:108E300080B2608388420CD94942401860832888F8
:108E40004549401C80B20B312880884201D3002064
:108E500028802D887D20C000618B68434018E06326
:108E600002903E48067828460A3800B226742085CB
:108E7000002803DA7D21C900401820853888302178
:108E80004843FCF7E0FB07462820205EFCF7D0FBB8
:108E90003946FCF7FDF97F21C905FCF7A0F9FCF77D
:108EA000FBFB2E4980B20880761E01E037E034E0FB
:108EB000B04201D101202073E5841620205EFCF72A
:108EC000C9FB074601910398FCF7D8FB244A254BC0
:108ED000FCF7CEFA05460E460298FCF7BBFB2A4685
:108EE0003346FCF7B7FA3A46019BFCF70FFAFCF75A
:108EF000E7FB2064A08B00F09DF868460088E083C3
:108F00000E480E495030807C607142006331084643
:108F10005130FCF733F90320207005B0F0BDFFF7A6
:108F2000CBF90000D4000020DE0000204800002023
:108F300000040050C9000020CA000020AC1100202D
:108F4000380D00200000002000D02724E40000207D
:108F5000F8000020A0140020E7030000DA00002041
:108F6000F853E3A59B843E4070B586B01421684653
:108F7000FCF71DF901250F4EED030022294630466E
:108F8000FDF7E3FC0120002401900294694600955E
:108F900003943046FDF714FC0320019002946946C7
:108FA000009503943046FDF70BFC022000F01CFFF7
:108FB00006B070BD0004005070470000F8B50446CC
:108FC00000206A461080194D55222A70AA226A7024
:108FD0000322AA70661DEE702A716971144A490055
:108FE0008918AC712246E81DFCF7C8F8002007E09C
:108FF00029186A468978128889186A461180401CA7
:10900000B042F5DB611DA81CFCF714FD0146684663
:10901000018029190078C871684640780872214695
:109020000931024800F0A2FAF8BD0000E013002068
:10903000380D002010B51A4CE08A228A61789042DF
:1090400001D3801AE08280B2628B034653435B18DF
:109050002383132802D1424350182083208B3021D0
:1090600048436421643048430E49E0620968401A6D
:10907000A062FCF7EFFA0C4A0C4BFCF761FAFCF724
:109080001FFB0B496062884202DD4A428018606221
:10909000002801DA4018606206490968486110BD7D
:1090A000C400002088000020F853E3A59B843E40C4
:1090B000FF7F0000A0140020034A1168382389B202
:1090C00099430143116070470030014010B5FDF72E
:1090D00049FC10BD10B59AB034216846FCF767F81A
:1090E00014210DA8FCF763F81C2112A8FCF75FF807
:1090F0001B4801680324E402A143C21489180160DB
:10910000FDF728FE17480169A14301610620009080
:10911000FF200130029001200390102004900220D3
:10912000099040040B90000100240C900A946846BA
:10913000FEF70EF80F200D9003200E900F94109460
:10914000012111940DA8FDF7F1FE8120129003205A
:1091500080041890149412A8FDF736FE1AB010BDC2
:109160000070004040100240104801688215114311
:109170000160C1680E4A1140C16001680D4A11408A
:1091800001608168490849008160016801229204F8
:1091900091430160C168FD2212049143C160002126
:1091A00001610649044888607047000000100240D1
:1091B0000C40FF88F6FFF6FE0050000800ED00E0CE
:1091C00070B501F089F8234C234DE06402E001F012
:1091D00083F8E064A842FAD1207801260525F60339
:1091E0002D07002806D001280CD0022817D003280C
:1091F0002CD129E0012231462846FDF7A6FBFFF7D6
:109200006BFD06E0012231462846FDF79EFBFFF785
:1092100043FB002231462846FDF797FB16E0A07A73
:109220000122401EA07231462846FDF78EFBFCF756
:10923000B1FD002231462846FDF787FBA07A0028C1
:1092400004D10120207001E0FFF744F800F036FF60
:1092500070BD0000480000203001CADE10B5818CCE
:10926000C90707D001684A6801235B049A43836AEF
:109270001A434A60818C890707D501684A6801232F
:109280001B049A43C36A1A434A60818C490707D575
:1092900001684A6801239B049A43036B1A434A609E
:1092A000818C090707D501684A680123DB039A43CB
:1092B000436B1A434A60818CC90607D502689168DE
:1092C00001231B039943836B19439160818C8906A9
:1092D00007D501688A6801235B039A43C36B1A436D
:1092E0008A60818C490612D503685A6801210905F4
:1092F000046C8A4322435A60026C8A4207D1026896
:10930000516803235B059943436C19435160818C79
:10931000090607D501684A680123DB04806C9A437B
:1093200002434A6010BD0000F8B500260446C66737
:10933000FDF712FB054620680068124F000709D5AB
:1093400001212B46002249052046009700F054FADF
:1093500000280DD12068006840070BD501212B465D
:10936000002289052046009700F046FA002801D027
:109370000320F8BD20206067A067603426740020B9
:10938000F8BD0000FFFFFF01F8B5184CC826E078D3
:10939000002829D16079002826D101206071144D60
:1093A000686B002700281ED0686BC821081A15E0DA
:1093B0001048E168405C616988470F480A210088CD
:1093C00048430E490880E068401CE060E068C82817
:1093D00000DBE760696BC820401A761EE1688142B5
:1093E00001D0002EE4DC6771F8BD000030000020E1
:1093F00000000240700C0020D4000020E00000209B
:1094000070B5224CE07800283FD1207900283CD16B
:10941000012020711E4EF16900250906002933DA6A
:109420002156625791420AD1F06940062CD5A079A5
:10943000002829D0A5712089401C208124E0A17931
:10944000002903D1A0710A2000F0D5FC002020568D
:10945000CC2148430F494218206912181279B26290
:10946000401C00222061A256CC235A4389588142D5
:109470000ADC25612078401C207020780E2800D15D
:109480002570A078401CA070257170BD30000020B0
:10949000003801404801002010B5806A00220146D2
:1094A00040314A834A82FEF7E6F810BD70B5846AFF
:1094B000606FA56F2168896800260906002906DA11
:1094C000212804D152200653204600F047F8206896
:1094D0008068400606D5222D04D15A200653204626
:1094E00000F02CF8E06F10210843E0672046FEF7FB
:1094F000C2F870BD10B501460968806A096889061E
:1095000014D400225A210A5201680A68FF23013349
:109510009A430A6001688A68520852008A600168AA
:109520008A6840239A438A6020218167FEF73EFAC9
:1095300010BD10B5806AFEF73AFA10BD01680A68DE
:10954000FF2321339A430A6001688A685208520057
:109550008A602021816700210166704701680A68DE
:10956000C0239A430A6020214167704770B5164CAA
:10957000E278002A0CD12279002A09D10122E27076
:109580000025C82903DC0222A256002A01DCE5706E
:1095900070BD0123E356CC2253430C4AD150012322
:1095A000E356CC2673439B180A460146181DFBF769
:1095B000E5FD6078401C607060780E2800D1657011
:1095C000A078401EA070E2E7300000204801002093
:1095D000F8B504462669A268E76932436669102037
:1095E00000253E432368324378491E68784F3E4049
:1095F00016431E6023685A6803263603B243E668A2
:1096000032435A602368A2698B4201D0266A3243F2
:109610009E680B273F02BE4316439E606D4E236833
:109620006D4AB3420CD1D2689207920F06D0012A3C
:1096300038D0022A34D0032A20D11EE001201DE0B8
:10964000664EB3420AD1D2680C26324026D0042A94
:1096500028D0082A24D00C2A10D10EE08B420DD13C
:10966000D66803229202164018D001229202B61A3E
:1096700018D0B61A14D0964200D10820564A0126B6
:10968000403A574FF6038B4236D100280CD00228BF
:109690000DD0042812D008281FD11CE00020EDE7CF
:1096A0000220EBE70420E9E7FDF7F6FC08E010688C
:1096B000C00601D5384605E04A4803E0FDF70CFD39
:1096C000002873D0626851005118814205D81103F7
:1096D000814202D303E03046F4E7012566E0010E43
:1096E00006025008002330185941FBF717FD0321EB
:1096F0000902411A3C4A55E0E169B14232D1030006
:1097000000F083F909070A0D06250606062B060058
:10971000E3E7FDF7C1FC1CE0FDF7CEFC19E01068A3
:109720006168C00602D54808304A01E0304A48085E
:109730008018FBF7DDFC80B201462E4A10399142B9
:10974000CBD8511C01400007400F08432CE0FDF727
:10975000C3FC616840004A08EAE7616801224808E2
:109760001204E5E7030000F050F909070A0D062688
:109770000606062C0600B0E7FDF78EFC1DE0FDF79F
:109780009BFC1AE010686168C00602D54808C01941
:1097900002E014484A081018FBF7AAFC80B2014600
:1097A000144A1039914298D82168C8600020206678
:1097B00060662846F8BDFDF78FFC61684A0880188E
:1097C000EAE7616848088019E6E7000000480040C1
:1097D000F369FFEF003801404010024000440040B0
:1097E00000093D000024F400FFFC0F0000127A0085
:1097F0000048E801EFFF0000FFB581B017460E46B4
:1098000004460A9D09E0681C07D0FDF7A5F80499F5
:10981000401AA8420CD8002D0AD02068C1693046F1
:10982000884318D00020B842EDD0002005B0F0BD2C
:1098300020680168FF22A13291430160206881689D
:1098400049084900816020206067A06700206034DB
:1098500020740320EAE70120E5E7000010B5044981
:109860001020096808620248FDF706FF10BD0000DD
:109870002815002001490D20887070473000002015
:1098800010B507480A22018A51438183FEF7E6FB9F
:10989000FEF7C8FCC82203490348FEF72BF810BDA9
:1098A000C4000020700C002028150020F8B53E4CA4
:1098B000002321783D4A1D46082910D0072947D0AA
:1098C000062950D0052952D0042953D0032954D059
:1098D000002956D0012958D002295AD05BE0A1783E
:1098E00000264A1F04E0314FBF5DFB189BB2761C77
:1098F0009642F8DB667927799A195118E3786278ED
:10990000C9188918C9194018C0430006000E1AD199
:10991000012E14D0022E16D125482449C018FBF779
:109920002DFC00F0C5FF642000F05EFABFF34F8FFE
:1099300021492048C860BFF34F8F00BFFDE7590899
:109940001046FFF73BFB2570E570A570A571F8BDCB
:10995000A1795054491CC8B2A071A178491F88420E
:10996000F5D1082001E0607007202070F8BDE0709C
:109970000620FAE760710520F7E7A070E570042083
:10998000F3E7552807D10120EFE7AA2803D10220E9
:10999000EBE7032803D02570E570A570F8BD032020
:1099A00020702071F8BD0000BB0000207C13002057
:1099B000380D00200400FA0500ED00E00FB410B5EA
:1099C00003A9044B044A029800F002F910BC08BC39
:1099D00004B018470DA60008080100202021020C41
:1099E00001D010211046020A01D0104608390209A0
:1099F00001D01046091F820801D01046891E420876
:109A000001D0881E7047081A704730B47446641E2F
:109A10002578641CAB4200D21D46635D5B00E318F1
:109A200030BC184702E008C8121F08C1002AFAD14A
:109A300070477047002001E001C1121F002AFBD1CE
:109A4000704708B50021684601706B46012202216B
:109A50002C2000F07BFD0221684601706B4601223C
:109A60002C2000F073FD08BD38B504466D20694612
:109A700008706B46012207492E2000F067FD064959
:109A8000002C01D0054A00E0054A2E2000F044FDDC
:109A900038BD000006080000061800000706000098
:109AA0000716000038B504466B4602220021362016
:109AB00000F018FCB3212300FFF7A7FF0E0F0815D5
:109AC0003A3A3A3A1C273A3A2F34483A0021684643
:109AD000017040784108490014E069460878800820
:109AE0008000401C04E06946087880088000801CE3
:109AF00008701DE0684602780A40483202704178DA
:109B0000802001436846417012E0684602780A40AE
:109B1000027040784106490EF4E769464878022110
:109B2000084303E069464878FD21084069464870CB
:109B30006B4601220021362000F008FD012200AB17
:109B400011463620013300F001FD38BD6946087822
:109B5000CF21084069462030CAE708B5032168468E
:109B60004170012101706B4602220021362000F075
:109B7000EDFC0122D20306212D2000F0CDFC0120B6
:109B800000F032F90120FFF78DFF08BD08B5020A89
:109B900069464A7008706B46022204212D2000F0AD
:109BA000D5FC0320694608706B46012206212D2052
:109BB00000F0CCFC0020694608706B4601220621AB
:109BC0002D2000F0C3FC0A212D2000F071FB08BD00
:109BD000FFB58DB00446002506E025280AD0109A6E
:109BE0000F999047641C6D1C20780028F5D12846F9
:109BF00011B0F0BD00270121484A009700E007435B
:109C0000641C23780846203B98401042F7D1207806
:109C10002E2817D1042007436078641C2A280CD111
:109C20000E98641C02C800910E900BE000990A2265
:109C3000514330394018641C009020780146303977
:109C40000929F3D920780028D1D0642808D06928C0
:109C500006D075281ED0109A0F9990476D1C5BE0B6
:109C60000A200E99019001C90E91002802DA4042A3
:109C70002D2102E0390504D52B216A4611720121FC
:109C800003E0F90704D02021F7E70BAE0B910DE0BC
:109C90000021FAE70A200E99019001C90E91F7E719
:109CA0000199FBF725FA3031761E31700028F7D183
:109CB00003A8801B20300190780701D5009801E0AF
:109CC000012000900199884201DD401A00E0002047
:109CD0000027009006E002A8109AC05D0F999047F7
:109CE0006D1C7F1C0B988742F5DB04E0109A302036
:109CF0000F9990476D1C0099481E00900029F5DCD3
:109D000005E03078109A761C0F9990476D1C0199E8
:109D1000481E01900029F4DC641C65E70928010055
:109D2000F8B54A002B4B520DD6182B4A0C46054667
:109D3000142E2BDA002E12DA284BFBF7E7FA00225A
:109D40001346FBF70DFE40D2002C03DA0124E40792
:109D500000253AE02046284337D0214C14E0214F1B
:109D60000B46F7403B402B4331D01C4BFBF7CEFA60
:109D700000221346FBF7F4FD27D2002C03DD01205F
:109D80000005F0400419BC4300251EE0332E1EDC04
:109D900033460027143BFF43DF40384217D00F4BB8
:109DA000FBF75EFB00221346FBF7DAFD0DD2002C19
:109DB0000ADD142E0CD03420811B0120884040196C
:109DC000A84200D2641C0546BD4321462846F8BD82
:109DD000641CF9E701FCFFFF9C7500883CE4377EBA
:109DE0000000F03FFFFF0F007D2110B5C900484380
:109DF00000F001F810BD002140E000BF00BF00BF2F
:109E000000BF00BF00BF00BF00BF00BF00BF00BF5A
:109E100000BF00BF00BF00BF00BF00BF00BF00BF4A
:109E200000BF00BF00BF00BF00BF00BF00BF00BF3A
:109E300000BF00BF00BF00BF00BF00BF00BF00BF2A
:109E400000BF00BF00BF00BF00BF00BF00BF00BF1A
:109E500000BF00BF00BF00BF00BF00BF00BF00BF0A
:109E600000BF00BF00BF00BF00BF00BF00BF00BFFA
:109E700000BF00BF00BF00BF00BF491C8142BCD370
:109E800070470000FEB50446002001900090607904
:109E9000734940000E5A61782578491E7148CFB247
:109EA0000163042D77D0072D75D000210291217810
:109EB00001736C49E379012292058969002B6CD00A
:109EC000914381616748217A4173217A82698907C8
:109ED000890B0A4382610021042000F028FB3246EE
:109EE00061492E2000F018FB3846FFF7BDFD5F4E9C
:109EF0000522705D810040185D49431807212B2021
:109F000000F024FB5B49029801220B180B2128204A
:109F100000F01CFB705D584980000A580C21282075
:109F200000F005FBE079554980004018A17949000F
:109F3000425A0221272000F0EFFA51487E00825B4E
:109F40000421272000F0E8FAE079002829D0A07841
:109F500004282CD0282069460872202206212720B8
:109F600000F0DAFA02AB01222621272000F0EEFAF7
:109F7000444938014018E1788900425808212720D7
:109F800000F0D5FAA17A601C627A0902114313D05D
:109F900016E000E001E0012188E71143F608816145
:109FA00090E764220621272000F0B6FAE0E71020AF
:109FB000694608720246D1E733490172090A4172C3
:109FC000417A007A0A0202432021272000F0A4FAF5
:109FD0002E4F0C2123203A6800F0A9FAF01982884C
:109FE0000421232000F098FAA07900280BD0E07912
:109FF0002749012243180021212000F0A7FA03205D
:10A000000190012000902A07120F1001024360788E
:10A0100000218007000B02430198000502430098CD
:10A02000400402432079C006400902436079C0061B
:10A0300002431F2000F07BFAA078617801230843D7
:10A0400002040848DB030261E179490319430A432A
:10A0500002610021082000F06AFA0020FEBD000025
:10A060007CA900080C0100200428000024A9000895
:10A07000010000201F0000202CA900084CA90008A6
:10A0800058A900085CA900084110000044A9000874
:10A090002100002038B50C4607498A8B0021024375
:10A0A0002C2000F039FA684604706B460122062124
:10A0B0002C2000F04BFA38BD0C01002010B5FFF742
:10A0C000C0FC10BD10B504460421362000F0F0F8A5
:10A0D0000121C902002C01D0084300E08843024658
:10A0E0000421362000F023FA10BD000038B54020CE
:10A0F0006946087000210E2000F0DAF804460022BC
:10A1000011460E2000F013FA6B46012200210D20AB
:10A1100000F01CFA074A00210F2000F008FA00F0B6
:10A12000E1F9224600210E2000F001FA0248002148
:10A13000017338BDF8FF27242C0100207CB50546AB
:10A140000420694608704B4C002060752146203180
:10A15000206348710873A0836063A06300F0BCF8BB
:10A16000454E206002E000F0B7F82060B042FAD11E
:10A170000020FFF797FC41480078242801D92438B3
:10A1800006E00621FAF7B4FF0622101A4001084340
:10A19000020601040A4301020A43024300211E2071
:10A1A00000F0C5F96B4601220021242000F0CEF911
:10A1B0001E20FFF7EBFC86B2300AA0730420FFF7E5
:10A1C000E5FC0006000E0DD002206946087101ABC7
:10A1D000012212212D2000F0B9F9A08B01210903E1
:10A1E0000843A08300F078F820600620FFF7CEFC3B
:10A1F00060600720FFF7CAFCA060F006C00E207563
:10A2000001D110202075C0B200F0DCF9E80707D0BA
:10A21000FFF7A3FCA08B0121C9020843A0830AE039
:10A220000521362000F02EF8154908400246052188
:10A23000362000F071F90120FFF734FC00210420E2
:10A2400000F036F8A0610021262000F031F8152139
:10A250008903084302460021262000F068F9002205
:10A260002621362000F058F900F036F82060002052
:10A270007CBD00000C0100203001CADE000000207F
:10A28000FFFD000038B5094C89B280B26B4602224E
:10A2900000F028F8002806D1684640780102684698
:10A2A0000078081884B2204638BD0000FFFF000087
:10A2B00038B50024E44389B280B26B46042200F032
:10A2C00011F8002806D103216846435C2202D41805
:10A2D000491EFAD5204638BD10B500210846FFF7C3
:10A2E000E7FF10BD38B5002909D0402420436C4653
:10A2F0002070C8B27F2906D8607002200AE0694643
:10A300000870012006E0802420436C466070C80974
:10A31000A0700320694600F0A5FA38BD10B51446B8
:10A3200003460A4621461120FFF7DCFF10BD10B599
:10A330000346052200211520FFF7D4FF10BD10B5FC
:10A340000346052200211720FFF7CCFF10BD38B5CA
:10A35000054600206946087000F0C4F8FF24013467
:10A360002246002D01D00322120200210D2000F010
:10A37000D3F8002D13D06B46012203210F20FFF7E5
:10A38000B1FF68460078000709D5FFF7AFFE224607
:10A3900000210D2000F0C0F80020C04338BD00208F
:10A3A00038BD10B5024601210A2000F0C0F810BDEA
:10A3B00010B5044600211A20FFF77AFF000D220392
:10A3C0000005120B024300211A2000F0B0F810BD66
:10A3D00010B5024602492E2000F09EF810BD000084
:10A3E00004180000F8B505466B460122032104203D
:10A3F000FFF778FF0126114C3607002D0DD02A46B5
:10A4000000210C2000F088F86946087810210843E4
:10A4100069460870A069304307E069460878EF2173
:10A42000084069460870A069B0430B46A06101224C
:10A430000321042000F08AF8F8BD00000C01002080
:10A4400010B502460021182000F066F810BD00008B
:10A45000F8B50746002568460570B807204C2E461B
:10A4600000280ADA8020694608706B460122002124
:10A470000D2000F06BF801202073F807694608787A
:10A4800021D006210843694608706B46012200214D
:10A490000D2000F05BF803210F20FFF7F3FE812170
:10A4A000C900084219D04020694608706B46012255
:10A4B00000210D2000F04AF80020FFF703FE0025E0
:10A4C0002673ED4309E002210843694608706B4694
:10A4D000012200210D2000F039F82846F8BD0000C7
:10A4E0002C0100201CB56B46012203210F20FFF731
:10A4F000F9FE684600784022C1091040C9014000B9
:10A50000814208D0012069460871024601AB03214F
:10A510000D2000F01BF81CBD08B56B461A70120A1E
:10A520005A7089B280B2022200F010F808BD38B526
:10A5300000236C46E254120A5B1C042BFADB89B23E
:10A5400080B22346042200F001F838BD38B58024DB
:10A55000002909D0C02528436D462870C8B27F293C
:10A5600007D86870022009E020436946087001207E
:10A5700004E020436870C809A8700320694600F011
:10A58000ADF938BD10B51446012312189B029A424A
:10A5900002D90020C04310BD0B46821E214609206F
:10A5A000FFF7D4FF002010BD10B5054A89051269D8
:10A5B00001430A4300210820FFF7B9FF002010BD26
:10A5C0000C01002038B504466B4601220E212B20D9
:10A5D000FFF788FE68460078E10640094001C90E91
:10A5E0000143684601706B4601220E212B20FFF7C4
:10A5F000ADFF38BD10B5002142541C06120A22439B
:10A600001B0A491C0429F7DB10BD000013B5012308
:10A610001A4669460248FDF7CBF900981CBD0000B8
:10A62000281500207CB5002425466846FFF77FFEEC
:10A6300004206946220E2D02154322020C5C1443AD
:10A64000401EF7D5204629467CBD7CB50024254612
:10A650006846FFF774FE04206946220E2D0215435A
:10A6600022020C5C1443401EF7D5204629467CBDCF
:10A67000FCF780F9FEF72EFDFDF704FD3749384859
:10A68000002522C005608561C56136490562C1604B
:10A690000838FCF78DFAFDF7E1FCFDF7C3FDFDF787
:10A6A0009FFDFDF7A7FC052601223607D1033046A2
:10A6B000FCF74BF9FEF77EFAFDF7A0FBFBF71AFA61
:10A6C000FBF7E8F90721B015FFF7E4FC264C0A2157
:10A6D000208A01224843A083170339463046FCF7FD
:10A6E00034F91F48C82221498830FDF703F9204E6C
:10A6F000207900282FD0FEF7EDFC2571FBF712FC26
:10A7000020700F2809D9012239463046FCF71DF97F
:10A71000FEF756FD0022394609E00122510330467A
:10A72000FCF713F9FEF74CFD0022012149033046E6
:10A73000FCF70BF9FDF7A6FAA08B002801D0401E0C
:10A74000A0830C48A18B00780843D1D10121084691
:10A75000FCF720FBCCE7FDF795FAC9E7007C004049
:10A76000A0140020FFFF0000C4000020700C002097
:10A77000000400503600002010B586B01748FCF7E2
:10A780009CF914216846FAF712FD15480090032041
:10A79000019000200290052069460007FCF710F8A0
:10A7A00069461048FCF70CF869460F48FCF708F8B2
:10A7B00001210846FCF7EEFAFF2401342046FCF79D
:10A7C000C1FA0A4908680422104308602046FCF7D1
:10A7D000C9FAFCF7CFFA06B010BD0000A0140020A3
:10A7E000FFFF00000004005000080050007000400F
:10A7F00010B50122920218491848FBF7F1F91648E2
:10A80000174902888A4225D0018004218180FF21D6
:10A81000F531C1800A21018100211E224181D243EC
:10A8200082810122C2810184018241828182C182AE
:10A83000018381831E23C3860223038778234387F2
:10A840008287C28702464032118451849184C18339
:10A8500000F02EF810BD0000380D002000FC0008AC
:10A86000AA550000F0B58C460025102605210907E1
:10A870008E620E4C08E067467F5DE760A768FF07C1
:10A88000FCD0E7681F706D1C8542F4DB0020074692
:10A8900006E0E760A568ED07FCD0E5681D54401CA4
:10A8A0009042F6D38E610020F0BD000000300140E0
:10A8B00070B572B60124074DA40221462846FBF765
:10A8C00075F9002804D0224603492846FBF712FAFE
:10A8D00062B670BD00FC0008380D0020F0B5002500
:10A8E000102605279C463F070B46BE620C4C06E02F
:10A8F000595DE160A168C907FCD0E1686D1C854223
:10A90000F6DB002007E06146095CE160A168C90749
:10A91000FCD0E168401C9042F5D3BE610020F0BD40
:10A92000003001400000010203040005405C00000B
:10A93000A05C0400C06C0800805C0400E03F1E00C6
:10A94000E07D1E0007A9022570889B880A0016007A
:10A95000010006000100020087008D002D001A3161
:10A9600052001A339A001A351D011A376B003B3119
:10A97000BE003B335E013B3596023B3700009959E0
:10A980009959EB518F421E45142E0080EB51F5284A
:10A990003333E13A703DE13AC235852BC23533336A
:10A9A000C235C235AE47E13A5138A33051380000C4
:10A9B0000000000000000102030406070809030468
:10A9C00006080C10182030000000000102030400EB
:10A9D000F0A90008000000200C010000249A0008E3
:10A9E000FCAA00080C01002044190000349A000859
:10A9F00000070400091E08054008260910400856F3
:10AA000008054008261D040008BE1D040008BED825
:10AA1000BC401008010000000000C8420000000017
:10AA20000000000000000000000000000000000026
:10AA30000000000000000000010000000000000015
:10AA400000000000000000000000000000005C1298
:10AA500000000000000000000000000000000000F6
:10AA600000000000000000000000000000000000E6
:10AA700000000000000000000000000000000000D6
:10AA800000000000000000000000000000000000C6
:10AA900000000000000000000000000000000000B6
:10AAA0000202040009090102008100000000000008
:10AAB0000100000000020000000000000000000093
:10AAC0000000000000000000000000000000000086
:10AAD0000000000000000000000000000000000076
:10AAE0000000000000000000000000000000000066
:0CAAF0000000000000002000000000003A
:04000005080050C1DE
:00000001FF
